:10000000C0710020711D0000C90500009D050000A1
:100010009D0500009D0500009D0500009D05000058
:100020000000000000000000000000009D0500002E
:100030009D050000000000009D05000089060000ED
:10004000E5170000111D0000000000000000000086
:1000500000000000000000000000000000000000A0
:100060000000000000000000000000000000000090
:100070000000000000000000000000000000000080
:100080000000000000000000000000000000000070
:10040000FFFFFFFFDFCEFFFFFCFF0F00FFFF0F002E
:10041000FCFF0F00FFFF0F00FCFF0F00FFFF0F00AE
:10042000FCFF0F20FFFF0F20FCFF7F40FFFF7F40FE
:10043000FCFF0D40FFFF0D40FFFFFFFFFFFFFFFF31
:10044000FFFFFFFFFFFFFFFFFFFFFFFFFFFFFFFFBC
:10045000FFFFFFFFFFFFFFFFFFFFFFFFFFFFFFFFAC
:10046000FFFFFFFFFFFFFFFFFFFFFFFFFFFFFFFF9C
:10047000FFFFFFFFFFFFFFFFFFFFFFFFFFFFFFFF8C
:10048000FFFFFFFFFFFFFFFFFFFFFFFFFFFFFFFF7C
:10049000FFFFFFFFFFFFFFFFFFFFFFFFFFFFFFFF6C
:1004A000FFFFFFFFFFFFFFFFFFFFFFFFFFFFFFFF5C
:1004B000FFFFFFFFFFFFFFFFFFFFFFFFFFFFFFFF4C
:1004C000FFFFFFFFFFFFFFFFFFFFFFFFFFFFFFFF3C
:1004D000FFFFFFFFFFFFFFFFFFFFFFFFFFFFFFFF2C
:1004E000FFFFFFFFFFFFFFFFFFFFFFFFFFFFFFFF1C
:1004F000FFFFFFFFFFFFFFFFFFFFFFFFFFFFFFFF0C
:100500000B4BC00030B5C4587F220D002000CBB289
:100510001540603011420AD0064ADB091B019B18C6
:100520005B1978331B7813B137335800201830BD6E
:100530008C2B0000D00500200122014B1A6070476F
:1005400000E100E00122034BDA67BFF34F8FBFF3F6
:100550006F8F704704E100E070B50500FFF7D0FF32
:10056000040060B12800FFF7EDFF03222388280074
:100570001340013A134323802280FFF7DDFF70BD53
:10058000054B80221900CC31088802430A801022D2
:1005900019880A431A8070470000094000BE70475E
:1005A000064B0749DA1DD27F1B6A920052585B0145
:1005B0005B0FDA401300034A1360704700E001400C
:1005C0009C050020B005002040F24012024B9A5AD0
:1005D000FE3392B25A86704700600040F7B5019032
:1005E000EFF31084012383F31088234A116819B9AB
:1005F000224BD9704031D97013680133136084F3F2
:10060000108800241E4E019B1B88A34212D8EFF3D2
:100610001081012383F31088136813B11368013B21
:10062000136012681AB9154BDA708032DA7081F3F0
:100630001088F7BD0199E3004968CB189D881F68B1
:100640002B0A0093FF231D4080235B021F420AD028
:10065000009B0C48190149198900735803407350D5
:1006600003003B407350009B01341B015B199B004E
:10067000F750A4B2C7E7C0463C110020000D04406B
:1006800000080440FFFFFEFF024A136801331360B5
:100690007047C046BC1100208A1892B240009142B7
:1006A00001D8824201DB121A92B210007047FFFF9C
:1006B000074A03001278824205D91820054A4343AD
:1006C0001068C018704700209A42FBD10248F9E731
:1006D000B8050020B4050020782A000010B5CB68CA
:1006E00002490B610121984710BDC046BC0500209E
:1006F000030010B5044A107813B1FFF71DFF10BDB9
:10070000FFF720FFFBE7C046980500200222024BBE
:100710005A8000221A71704768070020002210B525
:10072000024B1A80FFF7F2FF10BDC0466807002099
:1007300010B50020FFF7F2FF10BDFFFF8B790020FE
:1007400030B5012B21D1CB79022B1ED103008D783E
:10075000CC79022C10D19A4218D98C78AC4215D1A0
:10076000CC78844212D10C78013009191B198C798C
:10077000C0B29BB2012CEBD04A780020212A04D1D0
:1007800009338A7898B2024B1A7030BD0020FCE71A
:100790006807002070B50F26CB1D02003240D5B28D
:1007A0002C0000093034092A00DD07341C705A1E61
:1007B000994200D170BD1300EFE7FFFF030010B5B1
:1007C000094AC0339B009958084C214099509B58C6
:1007D000BFF35F8F1F22430910401E3A8240044935
:1007E00060339B005A5010BD00600040FFFFFEFFC9
:1007F00000E100E0F8B5FF260F4A83089B009B1834
:1008000004000322370040F200302240D200890168
:100810009740314091401D58BD4329431950200055
:10082000FFF7CCFF1F20012263090440A2400249C8
:100830009B005A50F8BDC04600E100E00022084B82
:100840001A719A78042A02D1013A9A707047072ADD
:10085000FCD11978013A4907F7D40232F5E7C046CE
:1008600068070020037810B5012B06D1034C2388BC
:100870001BB1FFF7E3FF0023238010BDF61000201B
:1008800083010001034340F2091018437047FFFF42
:1008900010B5002802DB024AFFF7ACFF10BDC046CE
:1008A00098110020F0B5194DAB686D689C6E2D78DD
:1008B000032D00D80134464246410EB9A0421BD355
:1008C0005B6BD2070BD4DB06DB0E032D09D91A09AB
:1008D0000123934360B9ABB902234B60F0BDDB0247
:1008E000F2E70C221340043B5A425341DBB2F1E7DA
:1008F000002BF1D10323F0E7032D01D90860EDE7C8
:100900000138FBE7002CE7D0F4E7C046981100203F
:10091000F0B514008618351B012C07D853085B006E
:10092000C0189A4201D003780B70F0BD6B782F7815
:100930001B023B430B80023CEDE7FFFF0323F0B5B6
:100940000B4085B007000D000093032B07D00C234C
:10095000304E0B4072681278062A02D123B905B0D6
:10096000F0BD0BB1032AFAD12B4B32689A42F6D173
:10097000B3685B6E0133BB42F1D301235B42029348
:1009800000232A00380002A90393FFF78BFFB26807
:10099000039B146B019373B940F2020C61462B0761
:1009A00001D504231900634602981D4221D08B0013
:1009B000D318D86418656B0604D58023106CDB034C
:1009C00003431364009B012B20D0144B1C40019B5C
:1009D0001B041C43022D13D1019B23B101223800BB
:1009E00002A9FFF75FFF0E4B1C40039B1B061C4335
:1009F00009E0009B5B1812339B00D3185860DAE7BC
:100A0000009B002BEFD1B3681C63A8E7022DE3D055
:100A1000E9E7C0469811002054504700FFFFFCFF53
:100A2000FFFFFFFCF7B50400019100891700628900
:100A3000A18883B295B2904225D3581B80B28142DF
:100A400027D80026320033003500381CAF4200D9C9
:100A5000281C85B22800013830D27F1BBFB257B1A5
:100A60003A1C9F4200D91A1C92B210003300013880
:100A700029D2AD18ADB221892A00A08889B2FFF72A
:100A80000BFE2081F7BD4800401B1818D6E75B1A03
:100A90009BB29942FBD9A94208D92668F218AB4209
:100AA00007D20026ED1AADB23300CEE76D1AADB213
:100AB000F1E7CD1A1B1AADB29BB2C6E701990978CE
:100AC00011700132C7E701990E781E700133CEE72D
:100AD000F7B504000191009200896289A58881B26E
:100AE00093B2904232D3CA1A92B2954206D24B1BAD
:100AF000A94200D24B192A009BB26381160017004D
:100B00001000002A28D16B461D88009B934200D913
:100B1000151CADB22A000199FFF7FAFE009B5A1B83
:100B200092B25AB1131CB24200D9331C9EB23200A9
:100B300038000199FFF7ECFEAD19ADB261892A00CA
:100B4000A08889B2FFF7A8FD6081F7BD6A00D21ABC
:100B50008A18C9E7491B89B28D42FBD99D4209D940
:100B60002768F818994208D8561BE91A9E19B6B298
:100B70008AB2C8E75B1B9BB2F0E700273E00C2E7E2
:100B8000F7B5224C0190E579A3792D021D432DB9CB
:100B9000012025706570A570E570FEBD019B2F1CBE
:100BA0005E331B885B065B0E00939D4201D96B464A
:100BB0001F88BFB297B1637822781B02A6781A43C8
:100BC000E378360416431B061E430199637A3A0004
:100BD00030001431DB070ED5FFF77AFF009B9F42F0
:100BE00002D20B4B019A5384ED1BABB21B0A0020BF
:100BF000A571E371D1E7F619FFF78AFE330A267073
:100C00006370330C360EA370E670E7E7D005002062
:100C10000080FFFF0C23F0B54B43414A85B09B1881
:100C20009A79DB7905001B0213430E000193A3B9E7
:100C300039B10B0044F2000237335B00595B1142BB
:100C4000FCD10C21002301204E43354AB354B61881
:100C50007370B370F37005B0F0BD40F200428BB218
:100C60001A43028402006432138003006C331B8831
:100C70009BB202932B8C1B071B0F9E42FAD16B8CED
:100C80009B04FCD56B46029A9F88019B934201D935
:100C90006B461F89BFB2EFB10C23734303930399D3
:100CA0001F4B8C462900039A1431D25C6344009395
:100CB0005B781B021A43009B9C78DB782404144366
:100CC0001B061C43009B3A005B7A2000DB0718D50B
:100CD000FFF7FEFE029B9F4201D2124B6B84002362
:100CE0002B842B8C1B07180F002BFAD10C21019B96
:100CF0004E43DF1B0A4BF618BBB21B0AB771F371E8
:100D0000A9E7FFF705FE064B039AE4199C54009AE5
:100D1000230A5370230C240E9370D470DAE7C04674
:100D2000D00500200080FFFFF0B51500384A85B0DF
:100D3000C30903939B18009001910833DA7F0024C4
:100D4000D20753D4334AD97F177801220A43DA777E
:100D5000314BFA003800D658FFF7F4FB009B002B0C
:100D600047D040F2204333842023328C1A42FCD0F7
:100D700001242A4B290A5A7A5971A2435A72FF2236
:100D80002A401A719A7132006032D9710292002D94
:100D900036D0019A1A70120A5A70019A120C9A707F
:100DA000019A110ED970009B63B1029B1C88E40B61
:100DB0005CB1330054331B8800241B0605D530007A
:100DC000FFF7DEFE0124029B1C803800FFF7B4FB16
:100DD00064B90F4A01219446039B63440833DA7FC8
:100DE0008A43DA77DA7F03318A43DA77200005B065
:100DF000F0BD009B33842023328C1A42FCD1B7E72C
:100E00001D705D709D70DD700523029A1380DCE714
:100E1000F4070020980500208C2B0000D00500204E
:100E200040B2C043002210B5C00F1100C001FFF74F
:100E30007BFF10BD70B5074D01000400082228009B
:100E400001F030FD0023AB60EB602078FFF7E8FF96
:100E500070BDC046BC05002070B505000024200010
:100E6000FFF726FCC8B14368280098470B4B0134B4
:100E70001B78E4B2A342F2D2094C3B2200212000AD
:100E800001F019FD1022FF21E01C01F014FD2000EB
:100E90001422FF21133001F00EFD70BDB8050020B3
:100EA000F407002010B5114B9889D989421A141CF7
:100EB00092B2402A00D940241A78A4B27F2A09D9D4
:100EC00088420FD022009968094801F0EBFC80208D
:100ED000074903E0884207D1002000212200FFF7E4
:100EE00023FF10BD8020F8E70020F1E7BC050020BB
:100EF000B4070020F8B5124E04000D0017000100E1
:100F00000822300001F0CEFC0023B560F381E379C4
:100F1000A2791B0213431A1CBB4200D93A1CB281AE
:100F2000E37991B2A2791B0213432BB109B12800D6
:100F30000DB1FFF7B7FFF8BD2078FFF771FFFAE7B3
:100F4000BC05002013B56C46227063701A0A1B0C96
:100F5000E3700023A2702171062269466371FFF7D6
:100F6000C9FF16BDF8B5058907894689040082883E
:100F7000ADB2BBB2B0B2B74207D31B1A9BB29A4212
:100F80001AD8E379DB09BBB9F8BD5600301A1B1833
:100F9000F4E7801A80B29042FBD2E28823685204C0
:100FA000520C5043181801F07DFC01222900A08842
:100FB000FFF772FB2081E7E72800ECE7F0B58DB082
:100FC000C14B00201C6823689847A589E3892289C2
:100FD000A8B299B29D4232D3431A9BB21D0093B17D
:100FE0009A4204D290422ED3811A89B2E1818A4278
:100FF0002CD9628963685204520C514309A85918CC
:1010000001F050FC0125E189208989B2AAB2FFF7DD
:1010100043FB2368E08101209847002D00D159E36C
:1010200009AC607801380728CAD801F05DFC1200CD
:101030001E00C9FF490349032700BF024C035300A8
:101040005B1AC318C9E7801881B2CFE7891A89B241
:10105000CDE72078FFF700FF142200219B4801F024
:101060002AFC22799A4B9A70AAE72078FFF7F4FEBF
:1010700014220021954801F01EFCA1E70120944FA5
:1010800004213B78602603433B703B000833DA7F42
:101090008243DA77DA7F8A43DA773B0028331A789B
:1010A00082431A701A788A431A702378874A019308
:1010B0000023136125792E40602E25D0402E0BD1C0
:1010C000844B0BB30100136101980AAA00E000BF32
:1010D000002800D074E717E0ED06ED0E012D00D1D9
:1010E000A2E1022D00D1C6E175B9202E16D1237AD6
:1010F0000F2B09D8764A9B18D878FFF7D9FA0AAA95
:101100000100002800D0D3E109AC00212078FFF7CE
:1011100023FA80212078FFF71FFA51E7002EF3D140
:1011200060790928F0D801F0DFFB70016801EFFF5A
:101130005F01EFFF0A00DF00EFFF16001C000AABA3
:1011400003CB03C20023614A9360D3603A78023331
:1011500013433B7034E77B7808AA911C0B70012283
:101160005EE1A37902937B78029A9A4205D1029BB1
:101170007B700AA8FFF75EFE22E77B787BB10198BF
:10118000FFF7E0F90A2140F20C0C013951BB01983C
:10119000FFF7D2F9BC780198FFF75EFEBC70029BA6
:1011A000002BE4D030223B784B4C93433B7001231F
:1011B000093403936378042BA6D10025464E2436C8
:1011C000361BB6B22800FFF773FA00289CD083685C
:1011D000320021000198984708286DD986426BD3C8
:1011E00000223FE063464B433C481B181E7A002E0A
:1011F000CBD07F250124019B3540394AF609DB001D
:1012000036019A5833185B1978331B7803959C4044
:10121000D08EA0431400D08660341BB11C0037343C
:1012200064001419002020809CB22500140068324C
:1012300064342580108062465343284A9B181872F4
:10124000039BB618F618783630709EE7A3782049CD
:10125000D318DBB25B18D978FF2900D054E70132EC
:10126000DD70D2B2039B9A42F0D12018A04214D86C
:101270001C4B1B78AB4200D246E7174B24339842F5
:1012800000D374E70122437803920B2B03D1C37878
:1012900003930378C01804008CE76378052B08D10A
:1012A000A2787A3313400A495B005B181333D209E2
:1012B0009D542378E418D9E70A4B01351B78EDB229
:1012C000AB4200D37EE71FE730080020BC050020BA
:1012D000F407002000000000B82A0000D00500201C
:1012E0008C2B0000B8050020E3881A0A501EDBB2E0
:1012F0000E2800D908E701F0F7FA0F001E002E00B3
:1013000007FF07FF6B001E0007FF07FF07FF07FF30
:1013100007FF07FF07FF15001222C9490AA8FFF7B8
:10132000E9FDD5E6C74B002B00D1EDE600E000BF9C
:10133000010018B9E8E6022A05D1C349CA788B78BA
:1013400012021A43EAE7C14A002A00D1DCE618007B
:1013500000E000BFECE77BB90222BD49BD4801F0C7
:10136000A1FA012040F20033FF2240000230BA49C6
:1013700003430B800240D1E7052B00D9C4E6B74AEE
:10138000B74C9B009F582378ABB9B64B21001B6824
:1013900058691D00FFF7FEF92100A8690831FFF721
:1013A000F9F92100E8691031FFF7F4F92100286A02
:1013B0001831FFF7EFF9380001F085FAA64AC0B2FC
:1013C000B042CFD9BC5D731C59008C52DEB2F7E736
:1013D000A54B002B00D197E600E000BF01000028DC
:1013E00000D191E6027899E7E388012B00D08BE6E3
:1013F0003A78073313433B70BBE6E388012B00D0F8
:1014000082E608223B789343F5E708AA911C012263
:101410003B78580910409B089218134003430B80F7
:101420000AA8FFF767FDCBE5237A0F2B00D96BE6FF
:101430008E4A9B18D878FFF73BF90100002800D1AD
:1014400062E601980AAAFFF749F9002800D0B7E53B
:1014500060236021227913400A4200D054E6627969
:1014600011000A39012900D94EE681490B610A2A87
:1014700000D07EE670E6237A02937F23029A1A4018
:101480000592092A00D93FE6029BDB09039353002A
:10149000764A07939B18039A9B18D87C0693FFF70C
:1014A00007F9049046B1002800D12DE601000AAAF0
:1014B0000198FFF713F90BE663791A00AA43012A92
:1014C0000CD0002B00D01FE6069F08AA0837FB7F30
:1014D000911C9B07DB0F2A000B80A1E7E288E2BB8F
:1014E000644A1578069A0832012B49D1D37F9B07AD
:1014F00033D528000299FFF703F80400F0B15E4BE2
:10150000EA002800D658FFF71DF840F200132380A8
:10151000039B13B1012323800DE0584A029B94469C
:10152000634478331A78330064331A80683633881A
:101530009B0B012BEED12800FEF7FEFF0221059B3D
:101540004A4A5B009B18039A9B180833DA7F8A4348
:10155000DA77DA7F01398A43DA77049B002B00D1EE
:101560002EE519000AAA0198FFF7B8F80023404AAF
:1015700013613B0028331B78DB0700D520E5F8E535
:10158000D37F9B07E9D402992800FEF7E5FF374A8D
:10159000079B9446039A63449B1802220833D97F21
:1015A0000A430121DA77DA7F0A43D5E77F222579DA
:1015B0002E492A4053005B18EF09DB191900012658
:1015C0000831C87FB043C877C87F0336B043C877B7
:1015D000002A69D12578A668254C2378DA09BA4211
:1015E00011D0002E00D0EBE4254B1BB121002800C8
:1015F00000E000BF2369002B00D1E1E403212800B3
:101600001B4A9847DCE47F2B07D8A068002800D14C
:10161000D6E432001B4901F045F9A268E38992192A
:101620009B19A260E2889BB2E3819A4201D03F2ECF
:1016300037D8236943BB2078FFF7F2FBC0E4C046EC
:10164000DC2A000000000000B82A000000000000B2
:10165000732A00006A06002068060020942B000010
:10166000401100209CB17F4000000000F4070020E2
:10167000BC050020980500208C2B0000D005002020
:1016800000000000B407002002212800124A9847F9
:1016900001000028CFD12800FEF75EFF802128003E
:1016A00039E5FFF7FFFB8BE4D87CFFF701F8030077
:1016B00080B11E69290062792078A368B0477FE471
:1016C000064B1B787CE46368002B00D178E4A068AB
:1016D000984775E40DB0F0BDBC050020F40700206C
:1016E00070B50B4C25680B4B1A7823685B1B632B7A
:1016F00008D9BFF34F8F084B084ADA60BFF34F8F0A
:10170000C046FDE7FF2AF0D0FFF758FCEBE7C046E4
:10171000BC1100209805002000ED00E00400FA054F
:1017200030B50400407885B0023803281FD801F096
:10173000D1F8025016220121274B1A788A431A70D9
:101740001A7849188A431A7000225A7004211A78AC
:101750008A431A70214B18684018210036E01E4B4E
:101760001A78D2070BD5042219780A431A701B4B3A
:1017700018680430F1E7184B1A78D207E6D405B0A0
:1017800030BD2800FEF794FF20B1436913B12078E3
:10179000616898470135EDB2114B1B78AB42F0D22E
:1017A0000D4B1A785207EAD504211A7801A88A430A
:1017B0001A7000210C2201F07EF86A46237801A9F4
:1017C000137105235371054B18680430FFF7CAFBEA
:1017D000D5E70025E0E7C046F407002030080020E8
:1017E000B8050020F0B58DB0EFF30383103B5BB27A
:1017F000C04AC0339B009958BF48014099509B583C
:10180000BE4EBF4FF38FDA0AD202D14308220A43F9
:101810009CB292B21BB2F287002B07DAF28F102330
:10182000120600D488E03A8813433B8063040ED547
:1018300009AD0C220021280001F03DF80523280005
:101840006B70FFF76DFF3B8EAE4A13403B86A304DF
:1018500011D53B8E9B040ED509AD0C22002128002A
:1018600001F029F8032328006B70FFF759FF3B8E26
:10187000A44A13403B86E30408D570232340202B61
:1018800000D1D3E05CD8102B00D175E0230529D519
:10189000E30700D4E6E00822F38F134222D044F29B
:1018A00000037B84984B07AD1B8800212B80974B4E
:1018B00004321B886B80964B1B88AB80954B1B8832
:1018C000EB8009235B42F38709AE300000F0F3FFA1
:1018D00006230822290073700AA800F0E3FF3000F5
:1018E000FFF71EFF630517D500218B4B1A8819805F
:1018F000D30711D58248FFF743F968B1874A09A891
:101900001179537940F20072099280221B020B4335
:101910000A920B93FFF704FFE3050BD5804AFB8E79
:10192000D18F1940CB439BB20291D387029B002BEE
:1019300000D0AEE00DB0F0BD3A889A433A8075E72A
:10194000602B05D015D860232340402B00D09DE7A5
:1019500009AD0C220021280000F0ADFF042328006F
:101960006B70FFF7DDFE42F200033A8E13433B86B5
:101970008CE7702BECD089E701237B87FB8644F250
:1019800000037B8400233B843B8C1B071A0F002B36
:10199000FAD13A843B8C1B07190F002BFAD1614A0C
:1019A0000133944660489A001218604801925A0028
:1019B00012185F489DB2058000206546288040F2DD
:1019C00000201080118040F2001201980133028043
:1019D000062BE7D1002155485A00554D121898B2F0
:1019E00028806046018040F2002001331080118081
:1019F0000A2BF0D198220021484800F05CFF072212
:101A00003B891340013B9BB2022B00D93EE7494A78
:101A10000021D55C09A80C2200F04DFF012306AA85
:101A20005373157409A8FFF77BFE2FE7424B1B8801
:101A30005B065A0E002B00D128E70021052307ADD5
:101A400029706B706A80A980E9800C2209A800F0D7
:101A500032FF062306AA5373290008220AA800F0C1
:101A600021FFDFE70726230033400193344200D0F3
:101A700038E73D8C1900AD06ED0FB540082209A8E6
:101A800000F019FF06AB5E731D74019B09A80B9350
:101A900026E7029800F032FF0C2343431F4C0190CD
:101AA0001B191A7AD209002A48D001001448FFF7FE
:101AB000B1F8002800D1B0E00C23019A09A85343E3
:101AC000164A9A1853791179D4791B0219439379DC
:101AD00024021C43157A0C1B0822002100F0EBFEA7
:101AE000072306AA5373157409A80B94FFF718FE71
:101AF00093E0C04600600040FFFFFEFF0200094087
:101B000000000940FFDFFFFF540009405600094074
:101B1000580009405A0009404A000940D0050020F9
:101B200008000940680009408C0009406E00094027
:101B300064000940702A000050000940019A002A00
:101B400000D187E09A79DB791B02134303936B463C
:101B50006A4A9B883B841380694B1B889BB2049321
:101B60003B8C019A1B071B0F9A42F9D17B8C9B047B
:101B7000FCD57B8C04991B051A0D8A4201D96B4652
:101B80001A8A93B205936B469D89039B91B28B424F
:101B900000D9151C0C23019AADB25343594AE15C9C
:101BA0009B185A789E7812021143DA7836040E4355
:101BB000120616433DB15B7ADB0735D52A003000AB
:101BC0005149FEF72FFF049BAB4202D944F20003B8
:101BD0007B8400233B843B8C1B07002BFBD1019AA9
:101BE0000C3303995A43481B4649521881B2090ADB
:101BF0009071D171049AAA4203D8039A05998A4236
:101C00000BD8019A3F4953430022E2545B185A70A3
:101C10009A70DA70002E00D04EE70123019A9340AB
:101C2000029A9A43029281E632002B00013B0DD2C8
:101C30000C23019A334853437219E254110A1B18BA
:101C40005970110C120E9970DA70BCE7397D117061
:101C50000132EBE7E279A37912021A432B4B03928C
:101C60001E887B8C76061B05760E1A0DB24200D9B3
:101C7000321C93B204936B469D89039B91B28B42B5
:101C800000D9151CADB285B1637822781B02A0780B
:101C90001A43E37800041B0610431843637ADB07FA
:101CA0001AD52A001849FEF7BDFEAE4202D944F209
:101CB00000037B84039B5A1B93B21B0AA271E3713E
:101CC000AE4203D8039B049A9342A6D80023237004
:101CD0006370A370E370EFE602002B00013B08D2B3
:101CE0004019030A20706370030C000EA370E070AB
:101CF000DBE7397D11700132F0E7C046640009402E
:101D00006C000940D0050020140009405E00094025
:101D100010B5FFF767FD10BD43F6B27310B5104A5A
:101D200010490400D1528168062000F039FE0E4BA4
:101D300010201B789B0703B1502000F029FE636838
:101D40001A7862B111241C572000FEF737FD1F22BC
:101D5000630914401E3AA24004499B005A5010BD2A
:101D600000C07E4080AAFFFFA0E0014000E100E04B
:101D7000F0B5E04BE04DE14A9D6040F2FE33E04EAD
:101D8000E049F2520022E04BE04C87B062801960DB
:101D9000DF49DA60596048F200011A619960FEF784
:101DA000FFFB40F280430122F254DA4BDA491A7801
:101DB00072B10A781AB9D9480278D207FCD51A78D4
:101DC000D206D00F002AFADB18701A78D206FCD49B
:101DD0000023D24A0B701378DB07FCD501260022C2
:101DE000CF4BC74F1E70CF4B3B62CF4BDA77FEF71E
:101DF000D7FB40F2FE334AF20052FA52E680E38803
:101E000099B2002BFBD102AA073201336380117013
:101E10001178EFF3108483F31088C44B598839B9D3
:101E200040F2FE304AF20256B54F395A3143395228
:101E30005988013189B2598084F31088EFF31084F6
:101E4000012181F31088BA4FBA4EB8683040B860AB
:101E5000B86884F31088B84C2068C007C00F1070B1
:101E60002068C007C00F10702068C007C00F107036
:101E7000EFF3108081F310888022BC685205224362
:101E8000BA60BA6880F31088EFF3108281F310888B
:101E9000598819B15988013989B259805B884BB981
:101EA00040F2FE310220964C635A8343A348034319
:101EB0009BB2635282F3108800244AF20053A04E72
:101EC000A04AB48033802B689F489A18B26041F2D0
:101ED0000002F3609D4B21005A8401239C4AB38089
:101EE000121A00F0E8FC9B489B4A9C49121A00F029
:101EF000D9FC9B4D9B4BED1AAD10A54200DD3FE296
:101F0000FEF74EFB0023984A984C994913701A002B
:101F1000185DC032920001335050202BF7D162B6C9
:101F2000944B954D95481D60FEF758FB40F2E83202
:101F3000934B1B68B3FBF2F38022013B52049342A4
:101F40000DD2C0218F4A6B485360036A09061B02F9
:101F50001B0A0B43036200239360073313600222C2
:101F6000894B8A499A6044F20002894B9A60894AF7
:101F700013688B4200D00AE240F2FE338649604883
:101F8000C152002111604AF20051C152834B844872
:101F90001D60844DFEF722FB2A68834B9A4264D071
:101FA000042300240121EB60804B29746B60804B7B
:101FB0006C61AB60EC61AC61EFF3108281F310886F
:101FC000FB683F318B43FB60FB6882F310884AF269
:101FD0000052AB6804A81A608022AB685204DC622D
:101FE000DC639C64DA62802212061A615A619A618B
:101FF00049F695025C629C62DC611C629A665A66D4
:10200000012301005B42220044F64B4004930594F7
:10201000FEF748FCAE68049B20007365B365059B22
:102020001A041B061A430192FEF72AFC3200AA2367
:102030008832DB03B4630121146033640323EA684C
:10204000F260019A706313430A43336320003263E2
:10205000FE31FEF71DFC21002000FEF719FC2100D7
:102060002000FEF715FC504B2B6003236A681178A3
:102070008B429B4144F61F615B425B18A9688B66EB
:1020800012781AB942F20F724A658A65CA6AD20793
:1020900005D44B66AA23DB030B64EB68CB600021FD
:1020A0000800FEF74BFC2B683F4A934202D1AB6815
:1020B000EA685A603F4C404B00226360230034338F
:1020C0001A700F4B07201A6A2D4B1968130E0D005A
:1020D00003409D402B00120F0240D3403748384A3E
:1020E000E360834274D8934272D0364883426FD003
:1020F00035486BE000ED00E00000000003A5FFFFA5
:1021000000E00140006CDC029C050020FEC00140A4
:1021100000127A00A0E0014036E001403CE00140BE
:1021200031E001400001001007E0014034110020BF
:10213000FC6F0440FFFFFFEF0008044000A5FFFF15
:10214000000D004000E0FFFFB0050020FE600040F1
:10215000C0110020000000209C050020AC2B0000D6
:102160009C0500209C05002028400440142B000002
:10217000006000408C11002054524F50F82A00009B
:10218000B005002010E000E06000044035817307D6
:1021900000000440F07F002002A5FFFF8411002012
:1021A000642B000098110020545047006C2B000055
:1021B00000820740FC100020002B0000FF083D00BB
:1021C00040420F0080841E00C0C62D00834250D1C3
:1021D000A648A74D006A5B194001400F8140C140ED
:1021E000B3FBF2F34919B1FBF2F1E36040F2835320
:1021F00006204B43B3FBF0F3236140F276334B43AD
:10220000B3FBF0F3636158234B43B3FBF0F3A361DB
:10221000984B00224B43B3FBF0F3E361964B974D91
:102220004B43B3FBF0F32362954BA1604B43B3FBED
:10223000F0F3636243F6C073EA54924B1A78012AB2
:1022400003D001221A7000F0ABFB8F48FFF764FD4A
:1022500040F2D8111F20E3685A1E6B58024020300C
:102260008343134388486B5000F06AFB08B9874BDF
:102270002360874E844800F073FB3378FF2B59D1DD
:102280003B220021834800F016FB0022824BDA81BA
:102290009A81824A1360824B23B1824800E000BFDA
:1022A000814B186000242000FEF702FA002841D07C
:1022B000036898477B4B01341B78E4B2A342F2D207
:1022C000002333707B68794A134040F200427B6000
:1022D000774B19880A431A801A885205FCD52021A9
:1022E000012005241A8840F200458A431A801A8882
:1022F00049188A431A801A887F2702431A806D4A38
:10230000146010225C5994435C516B4D2C88BC4383
:102310002143002429806949CC87694C1C86588751
:10232000D886C98F090602D519880A431A80002069
:10233000FEF702F9FEF724F944F61F673378FF2B06
:1023400001D0FEF73BFE5F4B5F491A680B68D21A5B
:10235000632AF3D95D4D64332C680B6020000021A3
:10236000FEF7ECFA5A4B1A78002A73D040F2CF727B
:1023700094426BD800221A7040F2D0732B60DDE7D4
:10238000544AA3009B181B6898470134B5E540F2F6
:1023900010433648C35CDB0708D440F2FE334E4896
:1023A000324CE0524AF200501160E05240F2F31316
:1023B000444801689942FCD940F2000C40F2FE33D7
:1023C00064462A484449C152146002004AF200504F
:1023D000D05244F200021068000E202800D0D5E54B
:1023E0002248C152EFF310810120019180F310883F
:1023F00079680C0040F60001214379607968019901
:1024000081F31088EFF3108480F3108841F200010B
:10241000786801437960796884F310884AF2005043
:102420001249C8526346B38072B6BFF34F8FBFF3F1
:102430006F8F6146294B1960294B9A60136883F3AB
:10244000088844F204031B6898479FE5254BE4186D
:102450002C6073E740F2D072A4182C60BC4200D804
:102460006CE701221A7044F6206387E700E0014020
:102470003F420F00B86A0500D066050000C07E40EC
:1024800068ED220090C07E40FC1000204E45504F69
:1024900098050020F407002088050020300800205F
:1024A00000000000B8050020B4050020FFF7FFFF82
:1024B00000000940F00009405E00094002000940A8
:1024C00000DDFFFFBC110020B81100209411002096
:1024D000F81000209C05002002A5FFFF10E000E09E
:1024E00000ED00E030F8FFFFF8B52F4B2F4C1A88B5
:1024F00044F200035209D202D218230000203433E0
:10250000187080202A49C002824205D240F600039A
:10251000200000F02DFAF8BDE26240F600022263CE
:102520006268A16212780AB101221A701F48FFF78F
:10253000F3FB01221F4D204E6B79204F93436B71AB
:10254000E36A1F4A9B181A0C9BB272827381A36ABA
:102550001B787B6381236B7563681B78002BDAD152
:10256000182312226169114800F0F2F9C0B9A16A7A
:102570004B1CA362E36A5A1CE262226B013A22639B
:1025800052B1104A9B181A0C9BB2728273814B781D
:102590007B6381236B75E3E7044800F0D1F9BAE768
:1025A0000828DDD0B7E7C046F4080020FC10002062
:1025B000F6080020FFC07E40FEC07E40FCC07E408A
:1025C0000000F0BD0100F0BDF7B5160013781F2222
:1025D0000F001A40012A00D051E11C005F32144064
:1025E00013421CD173780A2B0FD00B2B00D0E7E0DD
:1025F000012901D00124E3E0B278A24B5A70FEF722
:1026000085F83000FEF716FC07E00129F2D13A0008
:102610009C4901313000FEF76DFC0400D0E0202C15
:1026200000D02CE17078062800D928E100F052F99A
:10263000043C1C6B0E130E00012903D13000FEF781
:10264000F9FBD7E70329D5D1FFF74AF80129D1D102
:10265000FEF75CF8F2E70129CCD18A493A00300054
:102660000231FEF747FCC5E70129C3D1854A0223A1
:1026700011780C001C40194200D1A1E0F579B37922
:102680002D0200241D43402D00D999E00C32140086
:10269000F178B078090201432A006943200000F074
:1026A00001F92A002100B5E70129A3D175490B786A
:1026B0001C003C403B4200D182E08B78022B03D0CF
:1026C0000024052B00D07BE0F379B2791B020024B3
:1026D0001343402B74D801230B71F378B2781B029B
:1026E0001343CB80F379B2791B0213430B81F27948
:1026F000B37912021A431AB103238B700C3189E7A4
:1027000006238B707DE75F4DA978032906D0062943
:1027100000D182E0012F00D06CE784E0012F0DD1C1
:102720002A790521130022B16A780139130002B118
:102730006423EA783000FEF705FC6EE7032F00D033
:1027400058E72C790523002C00D196E00423E98872
:10275000AB704D4B2E8919800131FF31890140F258
:10276000C0730A001A40194211D172B6474F3B009C
:1027700034331A708022D202914223D2C90A40F621
:10278000000301223800C90200F012F962B62900E4
:102790003F4F404B38883200C0180C3100F082F8AF
:1027A0003B88F61840F60003B6B23E809E4205D143
:1027B00072B6FFF799FE62B600233B80FEF73EF843
:1027C0002000FEBD890A8A0201927A6812780AB155
:1027D00002221A702D48FFF79FFA01222E494B79E9
:1027E00093434B712D4B01989C463A63604440F2F1
:1027F00000418332B86200F0C3F87B681B78002B7D
:10280000C4D11122396A2148193300F0A1F80028F7
:10281000BCD11E4800F094F8B8E7012F06D12B79FF
:10282000022103B105310023EA7883E7032F00D0AA
:10283000E0E62C79022304B30723AB7072B6FFF7EE
:1028400053FE62B6FDF7FAFF0022104B1A60112208
:102850005B689A561300213300D1CBE61F21530940
:102860000A401E3991400A0020330D499B005A50FE
:10287000BFF34F8FBFF36F8FA2E7AB70BAE60024B0
:102880009EE7C04668070020F4080020FC100020E6
:10289000F6100020F6080020FFC07E400000F0BDCA
:1028A00000E100E0002310B59A4200D110BDCC5CDD
:1028B000C4540133F8E703008218934200D17047F3
:1028C00019700133F9E70023C25C0133002AFBD100
:1028D000581E704702B4714649084900095C490016
:1028E0008E4402BC7047C04603B47146490840009C
:1028F0004900095E49008E4403BC704741420840CC
:102900001C2101231B04984201D3000C10391B0A1F
:10291000984201D3000A08391B09984201D30009E3
:10292000043902A2105C401A7047C0461B1C1D1DD2
:102930001E1E1E1E1F1F1F1F1F1F1F1FFFFFFFFF2B
:1029400001B40248844601BC604700BFB1000020CA
:1029500001B40248844601BC604700BF6901002001
:1029600001B40248844601BC604700BF2D0100202D
:1029700001B40248844601BC604700BF290400201E
:1029800001B40248844601BC604700BF010000203A
:1029900001B40248844601BC604700BF89000020A2
:1029A00001B40248844601BC604700BF79000020A2
:1029B00001B40248844601BC604700BF09030020FF
:1029C00000000504342E352E30004275696C7420E9
:1029D000776974682052656E65736173204164760F
:1029E000616E63656420466C657869626C6520532E
:1029F0006F667477617265205061636B61676520F3
:102A000076657273696F6E20342E352E30004172F8
:102A10006475696E6F00536369656E6365204B6909
:102A2000742052332062302E3220444655004043F9
:102A30006F6465466C617368202F307830303030B9
:102A4000303030302F382A324B612C3132302A323C
:102A50004B67004044617461466C617368202F309D
:102A60007830383030303030302F382A314B6700F2
:102A70000100020904FFFFFF310700001D070000ED
:102A80003D070000C9250000000000000000000014
:102A9000040000000E00000004000000010300001C
:102AA0000000011307040000000001130E090000DC
:102AB000000001130F090000090224000101008039
:102AC000320904000000FE0102040904000100FEB6
:102AD000010205092107E80340000101120100027B
:102AE0000000004041236C01000101020301FFFFCF
:102AF000000001030103000005000000902A00000F
:102B00000000000065080000000000000000000058
:102B10000207020825260000000000000000000057
:102B200000000000000000000000000000000000A5
:102B30000000000001000000000000000000000094
:102B40000000000000000000000000000000000085
:102B50000000000000000000000000000000000075
:102B60000000000001000000F02A00000200000048
:102B700096980000020000004B4C000002FF00008D
:102B80000000000000000000342B0000000009409D
:102B900000000000732A00000E2A0000162A000020
:0C2BA000401100202E2A0000532A0000E3
:102BAC00431E59180A4B70B51C000126FF34657979
:102BBC00D2B2B54365711D00060CFE3580B26E8233
:102BCC00FC336881080C89B258626983627570BDE8
:102BDC0000C07E4082B00E4A0190136B5B060ED58E
:102BEC0000210C4B59750190136B5B06D80F002B11
:102BFC0008DA019B2BB1019B013B0193F4E7019B8C
:102C0C0013B9142002B07047019B013B0193E4E718
:102C1C00FCC07E40FFC07E404143032903D9890894
:102C2C0001390029FCD1704740F28013A521064AD6
:102C3C00D150C243054BD2B258705A7058705B7861
:102C4C00834200D1C046704700C07E40FFC07E402A
:102C5C0043F6B27344F6003273B5194E0400F35ABE
:102C6C0001929DB2012B09D19220FFF7DDFF0320C9
:102C7C00A168FFF7D1FF1220FFF7D6FF0820FFF75E
:102C8C00D3FF0620A168FFF7C7FF43F6B2720D4BC6
:102C9C00B352B35A98B253B9012D07D10A4BDD8008
:102CAC00DA8890B2002AFBD101325A8076BD019BA2
:102CBC001BB1019B013B0193EBE71420F6E7C046E7
:102CCC0000C07E4000AAFFFFFEC0014003000022AE
:102CDC00343310B51A7043F6B273094A0400D35A50
:102CEC000BB900F019FA0121064B20009A6A0A432D
:102CFC009A629A6A8A439A62FFF7AAFF10BDC0468D
:102D0C0000C07E40FCC07E40F8B5050008001600EF
:102D1C001F00FFF75FFF0400142804D12800FFF701
:102D2C00D5FF2000F8BD40F2F0133400044AD3580C
:102D3C001C401E42F5D02800FFF7C8FF3C00F0E70E
:102D4C0000C07E40002310B5934200D110BDCC5C76
:102D5C00C4540133F8E7002270B51C4B04005A80B0
:102D6C0043681A787AB111221F219A5653090A40E6
:102D7C001E3991400A00203315499B005A50BFF36D
:102D8C004F8FBFF36F8F43F6B273124A1249122062
:102D9C00D152FFF749FF0320A168FFF73DFF0F4B0E
:102DAC001B789B076BB10426C225D220C0B2FFF75B
:102DBC003BFFE8B2FFF738FF3000A168FFF72CFFAC
:102DCC0070BD062682259220F0E7C046FEC0014069
:102DDC0000E100E000C07E4001AAFFFFA0E001403E
:102DEC0013B50F4A0190136B1B0610D540F2DC1380
:102DFC0000240C49CC500190136B1B06D80F002BF0
:102E0C0008DA019B2BB1019B013B0193F4E7019B79
:102E1C000BB9142016BD019B013B0193E3E7C0469F
:102E2C00FCC07E4000C07E4070B50500406AFFF7D4
:102E3C00D7FF0400142804D12800FFF747FF200017
:102E4C0070BD40F2F013064AD258DF3B1400FF3B32
:102E5C001C401A42F3D02800FFF738FF1824EEE785
:102E6C0000C07E40F8B514000F0005001E00FFF7EF
:102E7C0072FF210083223800FFF792FE0334AB6906
:102E8C00A1085943102240F2F8132800FFF73CFF29
:102E9C0038B9044B2800DB6A1B07DB0F3370FFF7D4
:102EAC00D7FEF8BDFCC07E40F8B5040016000F003C
:102EBC001D00FFF750FF01210A4A380053798B435C
:102ECC002900537171438422FFF76AFEE1691923CB
:102EDC00112220007143FFF717FF10B92000FFF7F4
:102EEC00B7FEF8BDFFC07E40F0B585B0060002917C
:102EFC000392FFF730FF8323029C019301221E4FA4
:102F0C001E497B7913437B71039B03BB4FF6FF7305
:102F1C004B63CB6340F2DC13194A01993000D1505A
:102F2C00019B01330193FFF77FFF01227B790500A1
:102F3C0093437B7118B9019B0434872BDED130008D
:102F4C00FFF786FE05B90500280005B0F0BD6278D4
:102F5C002378120213434B63029BE31A0C2B07D109
:102F6C00029B039A987BDB7B1B0203431343D0E742
:102F7C00E278A3781202F9E7FFC07E40FCC07E40E5
:102F8C0000C07E4013B50F4C0A0C2300FE3389B2EF
:102F9C005A825981082201006846FFF7D3FE6B461E
:102FAC001A882300FC335A636A465288FF34DA636A
:102FBC006A4692885A646A46D2889A6481236375F9
:102FCC0013BDC04600C07E40F8B51D0004000E00C5
:102FDC001700FFF7C0FE0121ED0825630025134AF9
:102FEC00E762A66253798B435371236BBBB10DB16E
:102FFC002800F8BDE16AA06AFFF7C4FFA36A122299
:10300C000833A362E36A20000833E362236B21696F
:10301C00013B23631823FFF777FE0500E5E7002D3E
:10302C00E6D12000FFF714FEE2E7C046FFC07E4069
:10303C0030B50C4D0C4C52B940F2DC13800A890AA5
:10304C0080B289B260638232E163EA5030BD4FF6E0
:10305C00FF73E363013BFF3B1843812240F2DC1317
:10306C006063F2E700C07E40FCC07E40F8B51700FC
:10307C0005000C00FFF76FFE9FB140F2D812C02084
:10308C000321124E2140B358002783431C008901B1
:10309C000C43B4502800FFF7DBFD07B907003800DC
:1030AC00F8BD0126344063425C412002084C3900D3
:1030BC006379320033436371FFF7BAFF2800FFF7DF
:1030CC00B3FE63790700B3436371E3E700C07E404E
:1030DC00FFC07E40F7B501270E0004000C4D019295
:1030EC00FFF739FE6B7930003B436B71002201997D
:1030FC00FFF79EFF2000FFF797FE06006B7920007C
:10310C00BB436B71FFF7A4FD06B906003000FEBD92
:10311C00FFC07E400000000001B40248844601BCA0
:10312C00604700BF191D0000F106000034080020A4
:0C313C0010000C0000000000FF0000006C
:020000040101F8
:10001800FFFFFFFFFFFFFFFFFFFFFFFFFFFFFFFFE8
:0C002800FFFFFFFFFFFFFFFFFFFFFFFFD8
:0400000300001D716B
:00000001FF
